:1000000012C0189502C61895189518951895189548
:100010001895189518951895189518951895189578
:100020001895189518958FE58DBFC8E3E0E24E2E20
:1000300084E08EBFD4E0F4E05F2EA89584B7082E4C
:10004000877F84BF88E1992781BD91BDEEEFF3E002
:10005000A0E6B0E088278D933197E9F771DA66243E
:1000600086E886B980E087B9379AE2E8F0E080E474
:10007000AFDA58E0C895802DA5DA31965A95D1F7B8
:1000800004C020200E11110E2020E2EAF0E088E4E6
:100090009FDA58E0C895802D95DA31965A95D1F7B8
:1000A00004C0200E1111110A1B20E2ECF0E080E5E3
:1000B0008FDA58E0C895802D85DA31965A95D1F7B8
:1000C00004C004041F0404201F20E2EEF0E088E5D1
:1000D0007FDA58E0C895802D75DA31965A95D1F7B8
:1000E00004C0040404040404042078947BB77068FA
:1000F0007BBFA298A198A098A39AA49AA59A8A9A3D
:100100008D9A8E9ABA98BD988B98BB98BC98C29AD3
:10011000939AC59A8C9A949A8F9AB89AB99AC39AD4
:10012000C49AA898A998AA9885B7837F85BF08E341
:1001300016E820E030E0AFEAB0E00D931D932D9378
:100140003C93AFEBB0E0E2EDFEE17CDB0DE21EE3C1
:1001500025E030E0A3EBB0E00D931D932D933C938D
:10016000A4ECB0E0E8EDFEE16DDB06EC1DE624E377
:1001700030E0A7EBB0E00D931D932D933C93A9ECD9
:10018000B0E0EEEDFEE15EDB0AEB19E42CE032E0DC
:10019000ABEBB0E00D931D932D933C93AEECB0E030
:1001A000E4EEFEE14FDBB2D98CE012DA8FE711E02A
:1001B000BCD9EAEEFEE1A4D98FEB11E0B6D9EAEFA3
:1001C000FEE19ED9E2E0F0E0B2D9A0D98FE711E0DC
:1001D000ACD9ECE0FFE194D98FEB11E0A6D9ECE1CA
:1001E000FFE18ED9E2E0F0E0A2D906B348E30423B0
:1001F000A6EDB0E00C930091D600083109F001C0E3
:1002000048D684D9A4E6B0E0E0E0F0E094E0F7DD81
:10021000A8E6B0E0E4E0F0E094E0F1DDACE6B0E0C8
:10022000E8E0F0E094E0EBDDA0E7B0E0ECE0F0E047
:1002300094E0E5DDA4E7B0E0E0E1F0E094E0DFDDAC
:1002400082E08093D400E7EBF0E065DB88DBAAE88E
:10025000B0E0B6DBE2E9FEE1BCDCEAE8F0E05BDB63
:1002600025DCEDE0F0E0AAE8B0E0A9DDEAE8F0E0A6
:1002700014DBA2E8B0E0EDE0FF27A1DD82E080938F
:1002800080008CD58FE71CE050D9E2E2FFE138D93D
:100290008FEB1DE04AD9A4EDB0E00D91112745E0A8
:1002A00050E0C6DAAAEBB0E0A00FB11F23D981E07D
:1002B00080931701E6E9FEE18CDCEAE8F0E02BDB55
:1002C00027DCEDE0F0E0A8E7B0E079DD81E08093A5
:1002D0001801ABEDB0E08D919C91ADEDB0E08D9348
:1002E0009C93A7EDB0E08D919C91ABEDB0E08D9328
:1002F0009C9307B1007F006007B9A9DAA7EDB0E0D1
:100300008D939C93A7EDB0E00D911C91ABEDB0E007
:100310004D915C91040F151FA7EDB0E00D931C9358
:10032000A7EDB0E00D911C91ADEDB0E04D915C9169
:10033000040F151FA7EDB0E00D931C93A7EDB0E0DF
:100340000D911C9143E050E0B9D8A7EDB0E04D937A
:100350005C93A7EDB0E00D911C9142E350E0AED864
:10036000A9EDB0E04D935C93A1EEB0E08D919C912E
:10037000A3EEB0E08D939C93AFEDB0E08D919C9196
:10038000A1EEB0E08D939C9307B1007F016007B9A7
:100390005EDAAFEDB0E08D939C93E8E6F0E0C0DA72
:1003A000E8E7F0E0B8DA82DBEDE0F0E0ACE7B0E0FF
:1003B00006DDECE6F0E0B4DAECE7F0E0ACDAB7DB6F
:1003C000EDE0F0E0ACE7B0E0FADCECE7F0E0A8DA72
:1003D000EFEDF0E0D190E080FF240027C0DA10DBE1
:1003E000EDE0F0E0ACE7B0E0EADCECE7F0E055DAB5
:1003F000AFEDB0E0DD92EC92AFEDB0E00D911C916D
:10040000A1EEB0E04D915C91040F151FAFEDB0E08F
:100410000D931C93AFEDB0E00D911C91A3EEB0E0F5
:100420004D915C91040F151FAFEDB0E00D931C933F
:10043000AFEDB0E00D911C9143E050E03FD8AFED3F
:10044000B0E04D935C93A9EDB0E04D915C91AFEDC0
:10045000B0E00D911C910417150710F009F003C0CE
:1004600082E080931801A7EEB0E08D919C91A9EEF7
:10047000B0E08D939C93A5EEB0E08D919C91A7EE9A
:10048000B0E08D939C9307B1007F026007B9DFD97C
:10049000A5EEB0E08D939C93E0E7F0E041DAE8E769
:1004A000F0E039DA03DBEDE0F0E0ACE7B0E087DC68
:1004B000E4E7F0E035DAECE7F0E02DDA38DBEDE008
:1004C000F0E0ACE7B0E07BDCECE7F0E029DAE5EE69
:1004D000F0E0D190E080FF24002741DA91DAEDE0EE
:1004E000F0E0ACE7B0E06BDCECE7F0E0D6D9A5EEED
:1004F000B0E0DD92EC92A5EEB0E00D911C91A7EE7C
:10050000B0E04D915C91040F151FA5EEB0E00D9386
:100510001C93A5EEB0E00D911C91A9EEB0E04D91B9
:100520005C91040F151FA5EEB0E00D931C93A5EE92
:10053000B0E00D911C9143E050E0C0D7A5EEB0E0D3
:100540004D935C93A9EDB0E04D915C91A5EEB0E0C8
:100550000D911C910417150710F009F003C080E0FD
:1005600080931801E7EDF0E0D190E080FF240027B0
:10057000F6D92BDA2F933F934F935F93E7EDF0E09B
:10058000D190E080FF240027EAD95F914F913F91FD
:100590002F918CDAEDE0F0E0ABEEB0E010DCEFEDA7
:1005A000F0E0D190E080FF240027D9D90EDA2F9314
:1005B0003F934F935F93EFEDF0E0D190E080FF2405
:1005C0000027CDD95F914F913F912F916FDAEDE0E8
:1005D000F0E0AFEEB0E0F3DBE5EEF0E0D190E080EC
:1005E000FF240027BCD9F1D92F933F934F935F93FA
:1005F000E5EEF0E0D190E080FF240027B0D95F91D4
:100600004F913F912F9152DAEDE0F0E0A3EFB0E08F
:10061000D6DBE4E6F0E084D9EFEDF0E0D190E080C5
:10062000FF2400279CD9ECD9EDE0F0E0AFEFB0E07B
:10063000C6DBEFEEF0E074D9EBEEF0E06CD968DAEF
:10064000EDE0F0E0A7EFB0E0BADBE3EFF0E068D96F
:10065000E7EFF0E060D95CDAEDE0F0E0A7EFB0E0C2
:10066000AEDBEAE9FEE1B5DAE7EFF0E054D9C8D94C
:10067000EDE0F0E0A7EFB0E0A2DBEFEDF0E0D1902D
:10068000E080FF2400276BD9A0D9E7EFF0E043D941
:10069000B7D9EDE0F0E0A7EFB0E091DBEFEFF0E0ED
:1006A0003FD9E7EFF0E037D9ABD9EDE0F0E0A0E6D5
:1006B000B0E085DBE7EFF0E033D9E7EFF0E02BD9EE
:1006C000F5D9EDE0F0E0ABEFB0E079DBEBEFF0E097
:1006D00027D9E3EFF0E01FD91BDAEDE0F0E0ABEF54
:1006E000B0E06DDBEBEFF0E016D9EEE9FEE171DA98
:1006F00079DA08F006C0ABEFB0E0EEE9FEE18CDAA3
:1007000008C0EBEFF0E0A3DBEDE0F0E0ABEFB0E032
:1007100056DBEFEFF0E004D9EBEFF0E0FCD870D956
:10072000EDE0F0E0A3E0B1E04ADBE0E6F0E0F8D88D
:10073000E0E6F0E0F0D8BAD9EDE0F0E0ABE0B1E00F
:100740003EDBE3E0F1E0ECD8E3E0F1E0E4D8AED961
:10075000EDE0F0E0A7E0B1E032DBE7E0F1E0E0D887
:10076000EBE0F1E0D8D8E3D9EDE0F0E0ABE0B1E0C8
:1007700026DBEBE0F1E06BDBEDE0F0E0ABE0B1E0DD
:100780001EDBA8E0B4E0AF93BF93E0E6F0E0C3D88F
:100790005AD711E001E0BF91AF9153DAE8E0F4E0FD
:1007A000A7E9B0E007DBA8E0B4E0AF93BF93E3E0D4
:1007B000F1E0B1D848D711E001E0BF91AF9141DA43
:1007C000E8E0F4E0AEE9B0E0F5DAA8E0B4E0AF9339
:1007D000BF93EBE0F1E09FD836D711E001E0BF9185
:1007E000AF912FDAE8E0F4E0A5EAB0E0E3DA8FE7D2
:1007F00011E09BD6E8E2FFE183D68FE711E095D6C2
:1008000000911801003009F004C0EAE3FFE178D656
:10081000A4C1023009F004C0E0E4FFE171D69DC13B
:10082000013009F09AC100911701013009F013C09D
:10083000E6E4FFE165D6A7E9B0E05CD682E0C2D687
:10084000EAE4FFE15DD6AEE9B0E054D681E0BAD685
:100850008BE490E0E9D600911701023081E009F0C5
:1008600080E08F9300911701033081E009F080E070
:100870009F91892B882309F4D9C0E0E6F0E050D895
:10088000E4E6F0E048D853D9EDE0F0E0AFE0B1E0C5
:1008900096DAEFE0F1E044D8EFE0F1E03CD806D999
:1008A000EDE0F0E0AFE0B1E08ADAE3E0F1E038D883
:1008B000E3E0F1E030D8FAD8EDE0F0E0A3E1B1E018
:1008C0007EDAE3E1F1E02CD8EFE0F1E024D82FD993
:1008D000EDE0F0E0AFE0B1E072DAEFE0F1E0B7DADE
:1008E000EDE0F0E0AFE0B1E06ADAE4E6F0E018D87D
:1008F000E0E6F0E010D80CD9EDE0F0E0A7E0B1E0E0
:100900005EDAE7E0F1E00CD8E7E0F1E004D8CED819
:10091000EDE0F0E0A7E0B1E052DAE3E1F1E000D889
:10092000E7E0F1E0F8D703D9EDE0F0E0A7E0B1E0CF
:1009300046DAE7E0F1E08BDAEDE0F0E0A7E0B1E0E5
:100940003EDAE7E0F1E0ECD7EFE0F1E0E4D7EFD812
:10095000EDE0F0E0A3E1B1E032DAE7E0F1E0E0D78A
:10096000EFE0F1E0D8D7D4D8EDE0F0E0AFE0B1E0CF
:1009700026DAEFE0F1E0D4D7E3E1F1E0CCD740D8DC
:10098000EDE0F0E0A3E1B1E01ADAA8E0B4E0AF9363
:10099000BF93E3E1F1E0BFD756D611E002E0BF918B
:1009A000AF914FD9E8E0F4E0A7E9B0E003DA0091B5
:1009B0001701023009F00EC083E004D6ECE4FFE139
:1009C0009FD583E0FFD5EEE4FFE19AD5A5EAB0E03C
:1009D00091D529C0E3E1F1E09ED7EEE9FEE1F9D837
:1009E00001D981E008F080E08F93E3E1F1E093D753
:1009F000E2EAFEE1EED8F6D880E010F009F081E0FE
:100A00009F91892B882309F408C0E0E5FFE178D5A0
:100A100080E0D8D580E0D6D506C0E0E5FFE170D50E
:100A2000A7E9B0E067D58BE490E0FED5009117010F
:100A3000043009F092C0A3E1B1E0E6EAFEE1ECD8AF
:100A4000EAEAFEE1C6D8E3E1F1E065D7D9D7EDE007
:100A5000F0E0A3E1B1E0B3D9EAE8F0E061D7E3E187
:100A6000F1E059D7CDD7EDE0F0E0A3E1B1E0A7D9AF
:100A7000E3E0F1E055D7E3E1F1E04DD7C1D7EDE098
:100A8000F0E0AFE0B1E09BD9E3E1F1E049D7E3E08A
:100A9000F1E041D70BD8EDE0F0E0A3E1B1E08FD970
:100AA000A8E0B4E0AF93BF93E3E1F1E034D7CBD556
:100AB00011E001E0BF91AF91C4D8E8E0F4E0A7E90C
:100AC000B0E078D9EEEAFEE184D8EFE0F1E023D798
:100AD000EDD7EDE0F0E0AFE0B1E071D9A8E0B4E02F
:100AE000AF93BF93EFE0F1E016D7ADD511E001E091
:100AF000BF91AF91A6D8E8E0F4E0AEE9B0E05AD9F2
:100B0000EFE0F1E008D7E2EBFEE163D86BD810F03C
:100B100009F001C00DC0E6E5FFE1F2D4EEE5FFE12A
:100B2000EFD4A7E9B0E0E6D4E2E6FFE1E9D412C0F1
:100B3000E6E6FFE1E5D4AEE9B0E0DCD4EAE6FFE1C9
:100B4000DFD4EEE5FFE1DCD4A7E9B0E0D3D4E2E600
:100B5000FFE1D6D48BE490E067D506B348E30423E5
:100B6000A6EDB0E00C930091D600083209F013C056
:100B7000A7E1B1E08C918F5F8C9300911701043055
:100B800010F009F001C003C081E0809317018AEFE3
:100B900090E04AD52FC0003309F014C08091D400F2
:100BA00081508093D4000091D400013008F003C03C
:100BB00084E08093D40081E0809380008AEF90E00D
:100BC00033D518C0003209F015C0A4EDB0E08C9107
:100BD0008F5F8C930091D400043010F009F001C0B5
:100BE00003C081E08093D40081E0809380008AEF8D
:100BF00090E01AD500918000003010F009F001C09B
:100C000001C0CCD057CBF894FFCF0F921F922F92F8
:100C10003F924F925F927F92AF92BF920F931F933A
:100C20002F933F934F935F936F937F938F939F93F4
:100C3000AF93BF93CF93DF93EF93FF938FB78F93D0
:100C40007BB77F777BBF82E090E0EED406B348E3CA
:100C50000423A6EDB0E00C930091D600083109F012
:100C600023C0B29B10C0A4EDB0E08C918F5F8C9339
:100C70000091D400043010F009F001C003C081E0FD
:100C80008093D4000DC08091D40081508093D40013
:100C90000091D400003009F003C084E08093D400B8
:100CA00081E0809380005EC0B29B1EC0A2E8B0E0ED
:100CB0000D911D912D913C91A4EDB0E0AD90BB2420
:100CC000ABEAB0E0AA0CBB1CAA0CBB1CAA0DBB1D56
:100CD0004D915D916D917C91FCD7A2E8B0E00D93B0
:100CE0001D932D933D933BC0A2E8B0E00D911D9163
:100CF0002D913C91A4EDB0E0AD90BB24ABEAB0E007
:100D0000AA0CBB1CAA0CBB1CAA0DBB1D4D915D916E
:100D10006D917C91E3D7A2E8B0E00D931D932D93E4
:100D20003D93A7EBB0E04D915D916D917C91A2E870
:100D3000B0E00D911D912D913C91041715072607E8
:100D4000370708F00CC0A7EBB0E00D911D912D9175
:100D50003C91A2E8B0E00D931D932D933C9382E06B
:100D6000809380008F918FBFFF91EF91DF91CF91A2
:100D7000BF91AF919F918F917F916F915F914F91B3
:100D80003F912F911F910F91BF90AF907F905F90F7
:100D90004F903F902F901F900F90189500918000DA
:100DA000023009F060C0A2E8B0E00D911D912D91D4
:100DB0003C91A6E8B0E00D931D932D933C935A927D
:100DC0004A92A2E8B0E00D911D912D913C91D20183
:100DD0000D931D932D933C9384E026D5E3D2229668
:100DE00084E043D3A6E8B0E00D911D912D913C9194
:100DF000A2E8B0E00D931D932D933C93E2E8F0E060
:100E00008AD5ADD5AAE8B0E0DBD5E6EBFEE1E1D6C8
:100E1000EAE8F0E080D54AD6EDE0F0E0AAE8B0E0FC
:100E2000CED7A8E0B4E0AF93BF93EAE8F0E073D583
:100E30000AD411E003E0BF91AF9103D7E8E0F4E0FA
:100E4000AEE8B0E0B7D78FEB11E06FD3EEE6FFE18D
:100E500057D38FEB11E069D3AEE8B0E04BD3ECE7AA
:100E6000FFE14ED30FC08FEB1DE05FD3A4EDB0E0E8
:100E70000D91112745E050E0DBD4AAEBB0E0A00FC4
:100E8000B11F38D380E0809380007BB770687BBF50
:100E90000895A4E6B0E0E0E0F0E094E0B0D781E0AF
:100EA0008093AC000091AC00023010F009F001C05A
:100EB00003C081E08093AC0084EF91E0B5D3009152
:100EC000AC00013009F072C021D38FE711E02DD3BF
:100ED000E2E8FFE115D38FEB11E027D3E2E9FFE170
:100EE0000FD3A8E0B4E0E4E6F0E015D5ACD300D32E
:100EF00081E068D306B348E30423A6EDB0E00C9389
:100F00000091D600083009F002C000D349C000911A
:100F1000D600003309F00FC0EAEBFEE15AD6E4E652
:100F2000F0E0F9D4F5D5EDE0F0E0A4E6B0E047D785
:100F30008AEF90E079D30091D600003209F011C019
:100F4000A4E6B0E0EAEBFEE144D6E4E6F0E0E3D468
:100F5000EED5EDE0F0E0A4E6B0E031D78AEF90E026
:100F600063D3E4E6F0E0D7D4EEEBFEE132D63AD636
:100F700010F009F001C005C0A4E6B0E0EEEBFEE120
:100F80004BD6E4E6F0E0C7D4EAEBFEE122D62AD65F
:100F900008F005C0A4E6B0E0EAEBFEE13DD695CF4F
:100FA000ACEAB0E08C918F5F8C93A8C1023009F05D
:100FB000A5C1E7EBF0E0AFD4D2D4AAE8B0E000D509
:100FC000E2ECFEE106D6EAE8F0E0A5D46FD5EDE06C
:100FD000F0E0AAE8B0E0F3D6EAE8F0E05ED4A2E8F8
:100FE000B0E0EDE0FF27EBD682E080938000D6DE14
:100FF00007B1007F006007B92AD4A7EDB0E08D9358
:101000009C9307B1007F016007B921D4082F192FE5
:1010100042E050E00DD4AFEDB0E00D931C9307B16A
:10102000007F026007B913D4082F192F42E050E067
:10103000FFD3A5EEB0E00D931C938FE711E075D2BE
:10104000A8E0B4E0E5EEF0E05CD652D2E8E9FFE1DA
:1010500057D2A8E0B4E0EFEDF0E053D649D2E8E98A
:10106000FFE14ED2A8E0B4E0E7EDF0E04AD640D28E
:1010700088EC90E0D9D206B348E30423A6EDB0E0B3
:101080000C930091D600083009F004C08CE291E086
:10109000CBD201C0ADCFE7EBF0E03DD460D4AAE8FD
:1010A000B0E08ED4E6ECFEE194D5EAE8F0E033D48B
:1010B000FDD4EDE0F0E0AAE8B0E081D6EAE8F0E0A7
:1010C000ECD3A2E8B0E0EDE0FF2779D682E0809390
:1010D000800064DE8AEF90E0A7D207B1007F006055
:1010E00007B9B5D3A7EDB0E08D939C9307B1007F0E
:1010F000016007B9ACD3082F192F42E050E098D314
:10110000AFEDB0E00D931C9307B1007F026007B90B
:101110009ED3082F192F42E050E08AD3A5EEB0E00D
:101120000D931C93E7EDF0E0D190E080FF240027C1
:1011300016D44BD42F933F934F935F93EFEDF0E092
:10114000D190E080FF2400270AD45F914F913F9116
:101150002F9156D4EDE0F0E0ACE6B0E030D6E7ED0C
:10116000F0E0D190E080FF240027F9D32ED42F9314
:101170003F934F935F93E5EEF0E0D190E080FF2442
:101180000027EDD35F914F913F912F9139D4EDE03E
:10119000F0E0A4E7B0E013D6E7EBF0E0BCD3DFD398
:1011A000AAE8B0E00DD4EAECFEE113D5EAE8F0E0FD
:1011B000B2D37CD4EDE0F0E0AAE8B0E000D6EAE8F3
:1011C000F0E06BD3A2E8B0E0EDE0FF27F8D582E0D5
:1011D00080938000E3DD8AEF90E026D207B1007FA4
:1011E000006007B934D3A7EDB0E08D939C9307B1AD
:1011F000007F016007B92BD3082F192F42E050E080
:1012000017D3AFEDB0E00D931C9307B1007F0260E0
:1012100007B91DD3082F192F42E050E009D3A5EEDE
:10122000B0E00D931C93E7EDF0E0D190E080FF2457
:10123000002795D3CAD32F933F934F935F93EFED3E
:10124000F0E0D190E080FF24002789D35F914F9197
:101250003F912F91D5D3EDE0F0E0A8E6B0E0AFD517
:10126000E7EDF0E0D190E080FF24002778D3ADD304
:101270002F933F934F935F93E5EEF0E0D190E080A2
:10128000FF2400276CD35F914F913F912F91B8D3EA
:10129000EDE0F0E0A0E7B0E092D5ECE6F0E040D37E
:1012A000E8E6F0E038D334D4EDE0F0E0A8E6B0E0D2
:1012B00086D5EEECFEE18DD4E8E6F0E02CD3A0D3A9
:1012C000EDE0F0E0A8E6B0E07AD5E4E7F0E028D37E
:1012D000E0E7F0E020D31CD4EDE0F0E0A0E7B0E0E0
:1012E0006ED5EEECFEE175D4E0E7F0E014D388D3E0
:1012F000EDE0F0E0A0E7B0E062D501C0D3CD06D1CB
:10130000EAE9FFE1FDD0E0E0F0E0A4E6B0E094E03F
:101310007BE764D5E4E0F0E0A8E6B0E094E07BE7AA
:101320005DD5E8E0F0E0ACE6B0E094E07BE756D5D0
:10133000ECE0F0E0A0E7B0E094E07BE74FD5E0E13F
:10134000F0E0A4E7B0E094E07BE748D5E1E0F0E02E
:10135000EED008950895C09A81E08093190100911C
:101360001901083010F009F009C0979A9798A9E17F
:10137000B1E08C918F5F8C9308F4F1CFC09881E03D
:101380008093190100911901083010F009F009C08B
:10139000979A9798A9E1B1E08C918F5F8C9308F4AC
:1013A000F1CF0895C09881E080931A0100911A014D
:1013B000003210F009F025C000274427A881B98128
:1013C0008C9180FB00F94160042300FBA5EDB0E0A7
:1013D0008C9186F98C93A5EDB0E08C9186FBA8E307
:1013E000B0E08C9181F98C93979A979891E0A881BD
:1013F000B98140D2AAE1B1E08C918F5F8C9308F45F
:10140000D5CF81E080931A0100911A01083010F0C5
:1014100009F025C000274427A1E8B0E08C9180FBAB
:1014200000F94160042300FBA5EDB0E08C9186F942
:101430008C93A5EDB0E08C9186FBA8E3B0E08C9195
:1014400081F98C93979A979891E0A1E8B0E008D23F
:10145000AAE1B1E08C918F5F8C9308F4D5CFC09A4C
:10146000C0980895481A590A0895481A8827580AB2
:10147000089508D0DDD100FC10D0089503D01ED00F
:1014800001F8F9CF0024E89457FF02C009D068940E
:1014900000F80BD010F80124089502D009D0089567
:1014A000509540954F5F5F4F0895E89417FF08955A
:1014B000009510950F5F1F4F68940895352F242FC6
:1014C000E894452B11F468940895512F402F00277C
:1014D000112780E1440F551F001F111F021B130B22
:1014E000416018F4020F131F4E7F8A9599F70895F3
:1014F000A8E0B4E08D91882311F064D0FBCF08956B
:1015000064D3802D11F05ED0FBCF089581E060D0D0
:1015100014D080E85DC08FE7213039F08FEB2230A6
:1015200021F08FE8233009F08FEC810F51C088EE55
:1015300093E07AD03197D9F7089583E0992774C062
:101540008AEF90E071D08D9A8A9AA59AA49AA39A6C
:101550008E9A969885E090E067D0AB98959892988F
:10156000AD9AAC9AAB9AEF93FF93E4ECF0E050D0D5
:10157000FF91EF91AB9855D0AB9AEF93FF93E4ECCA
:10158000F0E046D0FF91EF91AB984BD0AB9AEF9340
:10159000FF93E4ECF0E03CD0FF91EF91AB9841D0A9
:1015A000AC98AB9AEF93FF93E4ECF0E031D0FF916D
:1015B000EF91AB9836D088E20BD08EE009D086E070
:1015C00007D00895969A829505D004D02AD0089520
:1015D0009698F9CF859510F4AC9A01C0AC98859592
:1015E00010F4AD9A01C0AD98859510F4929A01C09F
:1015F0009298859510F4959A01C09598AB9AEF93BF
:10160000FF93E4ECF0E004D0FF91EF91AB980895E4
:101610003197F1F70895689462F80895E89462F8B4
:10162000089581E090E000C0EF93FF93EE27E82B50
:10163000E92B31F0E0EDF7E03197F1F70197D1F7C1
:10164000FF91EF9108958DE207FD8D938F2D881FF7
:10165000802F881F8F57082F6894F7F8802F87FFF7
:1016600015C080958395082F80E38D938EE28D932E
:10167000802F815228F080E38D9399279C930895C1
:1016800044270A95802F09F192D01FC0805230F074
:101690009EE49D9381E48D939D93EFCF4427DF9249
:1016A000EF92FF920F938FE1801B11F0082F7FD0F4
:1016B00085D09EE29D930F91FF90EF90DF9044279D
:1016C0000395003209F4D7CF27D03F93EEE4F7E13A
:1016D00038E12F2D1E2D0D2DFF24EE24DD2444276F
:1016E000000F111F221F88F42F923F926ED2102CF0
:1016F0006CD2202C6AD2302C68D23197410DD21C8A
:10170000E31CF01C3F902F9001C0339631963A9520
:1017100039F73F9107D0B3CFDD0CEE1CFF1C0A95C3
:10172000D9F70895002719E058D08F93802B11F036
:10173000039501C08F911A95B9F7802F882309F47A
:101740009ACF8F91805D8D930A95D9F796CF0065DA
:10175000CD1D80B2E60E40597307A0ACB90350D638
:10176000DC01286BEE0094357700CA9A3B0065CD0A
:101770001D00B2E60E0059730700ACB90300D6DCB9
:1017800001006BEE0000357700009A3B0000CD1D94
:101790000000E60E000073070000B9030000DC0142
:1017A0000000EE000000770000003B000000F6940F
:1017B000E794D79447950A95D1F7089500270DD05F
:1017C0008F9303958F2D8E298D29842BC1F78F91AF
:1017D000805D8D930A95D9F750CF1F930F93002703
:1017E00010E2440FDD1CEE1CFF1C001F802F9AE04E
:1017F000890B10F0082F43951A9599F7802F0F91B8
:101800001F91089520931F013093200140932101DF
:1018100050932201089520911F01309120014091A1
:101820002101509122010895480E8827581E0895DD
:101830000F92B801469F8001479F100D569F100DD3
:101840000F900895C2D10D920020E1F70895369AC5
:101850003699FECF369A3699FECF84B195B1089568
:10186000903039F08C91869508F480689A95D9F774
:101870008C930895903081F00D911D912D913C91A4
:10188000369527951795079508F430689A95C1F70E
:101890003C932E931E930E9308953DD099271127C4
:1018A0008F2D880F80E8F82A802F881F08F41FEFFB
:1018B00041F08F57082F07FD04C0003240F08FEF32
:1018C00001C08827982FD82EE82EF82E09C08FE166
:1018D000801B082FF694E794D79497950A95D1F733
:1018E000112351F09095D094E094F09481E0980FFA
:1018F0008827D81EE81EF81E0F2DFE2CED2CD92EA1
:101900000895D094E094F09491E0D90E9927E91EBF
:10191000F91E10950895D190E190F19001910895EC
:1019200021913191419151910895102F90E8FF0C30
:10193000001F0927990FF7941078652F90E8440F3E
:10194000551F5927990F4795607800380895FF0C67
:1019500090E89027110F9795F794092F0895102F6D
:10196000BD2CDE2CEF2CF02E11234AF4B094D09431
:10197000E094F0949FEFB91AD90AE90AF90A0EE146
:10198000FF2039F4FE2CED2CDB2CBB240850C2F7D1
:101990006BC032F00A95BB0CDD1CEE1CFF1CF9CFAE
:1019A00001D0D5CFB7FE089590E8B91611F4D0FE56
:1019B00008959FEFD91AE90AF90A09F403950895E1
:1019C000DD92ED92FD920C930895502F2D2D3E2D1A
:1019D0004F2D612F08952DEC3CEC4CEC5DE3662718
:1019E0000FC099DFF2DFDD24EE2490E8F92E0FE33B
:1019F00007C096DF05C02227332740E251E466275F
:101A0000552351F1002381F190DF71F11627005821
:101A100050580894050B18F407FD03C025C007FDB6
:101A200023C0469537952795F694E794D79422D00E
:101A3000FF202AF0DD0CEE1CFF1C015073F09D2DE1
:101A4000969548F0DD203AF4EE202AF491E0D90E84
:101A50009927E91EF91E7BCF07C09FE7092FF92AB6
:101A60009FEFD92EE92E0895DD24EE24FF240027D0
:101A7000112708959F929924AA24BB2488E1D216A5
:101A8000E306F40628F0D21AE30AF40A089401C027
:101A90008894991CAA1CBB1CDD0CEE1CFF1C8A95AB
:101AA00071F7D92CEA2CFB2C9F9008953EDFE1F2D0
:101AB0005038D1F21627005850580894051F12F4D8
:101AC00018F4CBCF08F0D0CF0BD0FF202AF0BB0CFE
:101AD000DD1CEE1CFF1C3BCF0F5F0BF4BECF37CFDE
:101AE0009F929924AA24BB24992788E1990CAA1CC7
:101AF000BB1CDD1CEE1CFF1C30F4920EA31EB41E9A
:101B0000D91EE91EF91E8A9589F79F90089508DF6E
:101B10000CDF503829F090E869270CC00AF045D056
:101B200016CF5FE322273327442701C0F9DEFDDE0D
:101B30005038B1F3003899F3902F951B8BF312F4C2
:101B400034D0FACF983118F0222733274427983021
:101B500028F0232F342F44279850F9CF992329F0C8
:101B60004695379527959A95D9F7912F962742F064
:101B700014D0B0F6F794E794D7940F5F8BF66DCF3F
:101B800010D051F008F4BDDEFF2052F2DD0CEE1C47
:101B9000FF1C0150CBF761CF67CFD20EE31EF41EBE
:101BA0000895D21AE30AF40A0895DF92EF92FF92A1
:101BB0000F931F93D22EE32EF42E052F162F6F9125
:101BC0005F914F913F912F910895C89531960020D4
:101BD0000895FBDF202DF9DF302DF7DF402DF5DFF5
:101BE000502D089507FB00680EF40F7757FB5068DF
:101BF0000EF45F7707FD02C057FF05C0D216E3065B
:101C0000F406050708952D153E054F055007089564
:101C100091E005C092E003C094E001C098E0D5DFF8
:101C20000D929A95E1F7089599278D9193958823C0
:101C3000E1F7939511968C9311978E919A95D1F720
:101C40000895EA2FFB2F00244C918D9103948E323E
:101C5000E1F711248D9113948823E1F71A9410165B
:101C600040F41197202F2119239580E38D932A9515
:101C7000E9F7113039F59927AE2FBF2FA00DB91F05
:101C8000A00FB91F8C919C93853308F421C031E0DB
:101C90008E918E32E9F38D3241F0830F8A3319F43D
:101CA00080E331E001C033278C93AE1789F73323EB
:101CB00041F0AE2FBF2FB8DF81E34D3209F43196EA
:101CC000808308958827E00DF81FE00FF81F8083B8
:101CD0000895040F151F261F371F0895041B150BA9
:101CE000260B370B0895000F111F221F331F089575
:101CF00000951095209530950F5F1F4F2F4F3F4F48
:101D00000895019110810EC00191119121913081AE
:101D10000BC00191108117FF05C03FEF2FEF04C0EA
:101D2000008111272227332737FF03C0E1DF8DE22F
:101D30008D93CF93DF93CF92DF92EF92AA24BB24AF
:101D4000CC24DD24EE2440E2CAE0DD2755E093E315
:101D50008881890F87FD9F7083FD907F891B899300
:101D60005A95A9F7C0DFAA1CBB1CCC1CDD1CEE1CBD
:101D70004A9551F7E894EFE0FF2782910ED0EB30BF
:101D8000E0F71EF068948A2D0CD088278D93EF9091
:101D9000DF90CF90DF91CF910895982F829501D059
:101DA000892F8F70805D26F0803309F40895689440
:101DB0008D93089581918D938823E1F7089594E0A0
:101DC00081918D939A95E1F70895E199FECFEEBB4D
:101DD000FFBB3196089591E001C092E07B3751F44A
:101DE0007FB7F894F2DF8D918DBBE29AE19A9A95D4
:101DF000C9F77FBF7727089591E001C092E0E5DF42
:101E0000E09A8DB38D939A95D1F7089588E00FB637
:101E1000F8945A924A92E42DF52DA42DB52D480E32
:101E20008827581E0FBE08950FB6F8944990599010
:101E30000FBE089570DD802FFF0C001F901728F44F
:101E4000091B881F0795F79408950ECE0DCE63DD0C
:101E50000023E2F3D9F388E0DADFB2DD1196FF0C5C
:101E6000001F8FE7080F0795F7940695F79483E016
:101E70008F93ABDDA5DD13974EDDC2DD51DD3897C5
:101E800056DE91E0D8DF8F918A9511F08F93F1CFD4
:101E9000CBCF00000C42000080400000004000005A
:101EA0000000000020410000003FC3F5484000242E
:101EB000744900007A440000FA320000803F0000BC
:101EC000964300001B4300002042000087430000AF
:101ED000B841316B487A00002031306B000031305E
:101EE000306B0000314D487A000053503646524561
:101EF000202056532076312E3100687474703A2FAA
:101F00002F6C782D6E65742E706C000050726573A6
:101F10007320627574746F6E20746F00534554554E
:101F2000500046312020200020202020202020208A
:101F30002020202020202020000053484F52540011
:101F40004F50454E00005A3D00006A005A003D00C7
:101F50005357523D0000433E316E462000004C3D39
:101F6000000075480000433D00007046200020201E
:101F70002020202020202020202000004D487A20F2
:101F800000004D65617375726520726573697374C5
:101F90002E0052203D20000020005A61706973001D
:00000001FF
